:020000040000FA
:10000000850107309F00031383161F3085000030E1
:1000100086008601031383122A302A302A304A30A0
:10002000613072302E3043306C306F3063306B3063
:100030002E3032303030313036302E304D3061306D
:1000400072306930753073302E3054306130633027
:100050006930753063302E302A302A302A308601DC
:10006000A3013C30230203193C20230886004020D2
:100070008613A313A30A31288601A301A31708003E
:1000800047204720472047204720472008003A3094
:10009000A000A101A10B4A28A00B4A280030A00013
:1000A000A101A10B5128A00B51280030A000A101F3
:1000B000A10B5828A00B58280030A000A101A10BCB
:1000C0005F28A00B5F280030A000A101A10B6628CB
:0E00D000A00B66284D30A000A00B6C28080085
:0200DE000034EC
:0200E0000034EA
:00000001FF
